:104D8A000000090101240200000301FA0400FA05E7
:104D9A0000020A0A5A0B000F0C00FA0D00030E005B
:104DAA00030F0132100096120132130AFA1401029B
:104DBA0015000217010A18010A1905321A010A1BFD
:104DCA00010A1C053223011E2400642A00FA2B0062
:104DDA00FA2C50782D003C2E00462F001E3000641D
:104DEA003250783300003432FA35016436016437C0
:104DFA000150380A643C00643E003C3F000140FF19
:104E0A00FF411450420A5A430AC844053245007801
:104E1A004600FA4701224802034C00FA4EFFFF50AF
:104E2A000606510596520A32530B28540A96560121
:104E3A0002570546580002590A465A32FA5B010AD5
:104E4A005C0A325E000A5F00FE61FFFF64021067BF
:104E5A0001036A0A3C6B00006C32967801327901D0
:104E6A0032FAFAFA0000090101240200000301FAE9
:104E7A000400FA0500020A0A5A0B000F0C00FA0D88
:104E8A0000030E00030F0132100096120132130ABA
:104E9A00FA14010215000017010A18010A1905324D
:104EAA001A010A1B010A1C053223011E2400642A66
:104EBA0000FA2B00FA2C50782D003C2E00462F00C9
:104ECA001E3000643250783300003432FA350164FF
:104EDA00360164370150380A643C00643E003C3FA6
:104EEA00000140FFFF411450420A5A430AC84405D0
:104EFA00324500784600FA4701224802024C00FA7D
:104F0A004EFFFF500606510596520A32530B28549B
:104F1A000A96560101570546580001590A465A325F
:104F2A00FA5B010A5C0A325E000A5F00FE61FFFF5B
:104F3A006402106701036A0A3C6B00006C329678BF
:104F4A000132790132FAFAFA0065006F00790083BA
:104F5A00008D009700A100AC00B600C000CA00D4C2
:104F6A0000DE00E800F2005B0063006A0072007A6B
:104F7A00008200890091009900A100A800B000B841
:104F8A0000BF00C700CF00D600DF00E600EE00F643
:104F9A0000400046004C00520059005F0065006B5B
:104FAA0000710077007D00830089008F0095009CC6
:104FBA0000A200A800AE00B400BA00C000C600CC2F
:0C4FCA0000D200D900DF00E500EB00F190
:10009E00AE33AF34740A8E048F05FF1252428C3584
:1000AE008D36AE33AF34740A8E048F05FF12527B39
:1000BE008C338D34E53445336013740AC39534FFA5
:1000CE00E49533FE8E338F3478351252BDE550A849
:1000DE0035B80015D395364010E550C39536FFE47C
:1000EE009535FE8E358F368010E5502424C3953617
:1000FE00FFE49535FE8E358F36AE35AF3674236FF1
:10010E004E600674246F4E701AAE35AF3674236F80
:10011E004E70057550018003755002753622753587
:10012E0000800375500022900084E0B40104C20BDD
:10013E008002D20B900085E0B40104C20C8002D282
:10014E000C9000C2E075F0DCA4FFAEF0740A8E04D1
:10015E008F05FF1252429007AAECF0A3EDF0A20811
:10016E00401674038C068D0712526074011252529F
:10017E009007A8EEF0A3EFF07E017F00900080E0E4
:10018E001252609000C3E08E048F05FF125242742B
:10019E000AFF1252428D399000CCE075F0DCA4FFBC
:1001AE00AEF0740A8E048F05FF1252429007AEEC29
:1001BE00F0A3EDF09000CEE060139000CEE0F5F0ED
:1001CE00741684FF7E00EF9007B6F080067464907C
:1001DE0007B6F09000D6E0B4020674029000B8F0B4
:1001EE009000ADE0B40B0874E390006FF08049907E
:1001FE0000ADE0B419129000C3E0904F3D12008C98
:10020E00E49390006FF080309000ADE0B41E129039
:10021E0000C3E0904F5B12008CE49390006FF0806F
:10022E00179000ADE0B428109000C3E0904F8512F7
:10023E00008CE49390006FF090004BE0C394055057
:10024E002274019000C6F09000C8E0B4020674015A
:10025E009000C8F09000B8E0D3940240067402906B
:10026E0000B8F09000E0E0B40117900024740FF095
:10027E00A374FFF0900026E4F0A3F074029000E067
:10028E00F09000E0E0B40341900026E0FEA3E0FF12
:10029E00900024E0FCA3E0FD1252B57410125260DF
:1002AE007408125252EF90006CF0EF700674FF90CB
:1002BE00006CF074009000E0F0900025E090006D6E
:1002CE00F0900024E090006EF0900071E090003409
:1002DE00F0900034E0240C900035F0900034E024CF
:1002EE0018900036F0900035E0D39424400B900027
:1002FE0035E0C39424900035F0900036E0D394247A
:10030E00400B900036E0C39424900036F090003AF3
:10031E00E4F0900034E064236007900034E0B424ED
:10032E0020900034E0B42306740290003AF090005E
:10033E0034E0B4240690003A7401F0900034740155
:10034E00F090003BE4F0900035E0642360079000ED
:10035E0035E0B42420900035E0B4230674029000FA
:10036E003BF0900035E0B4240690003B7401F09011
:10037E0000357401F090003CE4F0900036E0642308
:10038E006007900036E0B42420900036E0B42306D7
:10039E00740290003CF0900036E0B4240690003CCD
:1003AE007401F09000367401F0900071E0FE900040
:1003BE00D4E02E90003EF09000AFE0B401609000CB
:1003CE003EE06412600790003EE0B4240690003ECA
:1003DE00E004F090003EE06411600790003EE0B44F
:1003EE00230690003EE014F090003EE0D3942440AB
:1003FE000B90003EE0C3942490003EF090003EE04F
:10040E00D39412400D90003EE0C3941290003FF042
:10041E00800A90003EE0241290003FF0807690001B
:10042E003EE0640C600F90003EE0641860079000A0
:10043E003EE0B4240690003EE004F090003EE064FE
:10044E000B600F90003EE06417600790003EE0B432
:10045E00230690003EE014F090003EE0D39424403A
:10046E000B90003EE0C3942490003EF090003EE0DE
:10047E00D3940C400B90003EE0C3940C90003EF0E1
:10048E0090003EE0D3940C400B90003EE0C3940CE1
:10049E0090003EF09000B7E0900037F0900037E00B
:1004AE00640B6007900037E0B41706900037E01435
:1004BE00F0900037E0640C6007900037E0B4180647
:1004CE00900037E004F0900037E0240C900038F0F4
:1004DE00900037E02418900039F0900038E0D39463
:1004EE0024400B900038E0C39424900038F0900024
:1004FE0039E0D39424400B900039E0C3942490004B
:10050E0039F022C293C294C291C292C287C290E5C0
:10051E00B554EFF5B5E5B554DFF5B5C296C295C243
:10052E00A0C297C2A2C2A1E5B554BFF5B5E5B554B8
:10053E007FF5B5E5B554FBF5B5C20D7537469000A0
:10054E00BAE07005754902800375490390000C747A
:10055E00FFF0A374DCF090009BE0900012F8E4F042
:10056E00E8A3F0C213C215C21774C8900028F07425
:10057E00C890002CF074C8900030F07526007525D8
:10058E0000C208756C00E54BB40903754B00753C51
:10059E000090001AE4F0A3F0754C1E752800752724
:1005AE0000C210C211C2129007AAE0FEA3E0FF74AF
:1005BE000312526074011252529007A8EEF0A3EF8C
:1005CE00F0C203900010E4F0A3F0C2222285F9508D
:1005DE0085FA517E017F00E551125260E5502FFFE2
:1005EE0050010E8E338F349007AAE0FCA3E0FDEF8E
:1005FE002DFDEE3CFC8C358D36E536F5FBE535F5FF
:10060E00FC22053D22A2D8B34006C296C295C2A0D6
:10061E0075D8402285A74F75A7109000B8E06403E7
:10062E0060079000D6E0B4022CA2D8B34002C29369
:10063E00A2D9B34002C294A2DAB34002C291A2DBA5
:10064E00B34002C292A2DCB34002C287A2DDB34025
:10065E0002C290801BA2D8B34004C293C292A2D908
:10066E00B34004C294C287A2DAB34004C291C290CE
:10067E0075D840854FA722900047E4936406600228
:10068E0080FE74C89007B0F8E4F0E8A3F075B500EA
:10069E0075840175A70075FF8075EF0690003DE427
:1006AE00F075C91075A70F75A1C775A70075D9008C
:1006BE0075CE0C75A70F75F1FE75F2FF75F3077504
:1006CE00F47875A4BA75A5FF75A60775AE0075AF5B
:1006DE00FF75D48175D5FF75D6FF75D7FF75A70049
:1006EE0075A20175A14775F80975D80075D90475FD
:1006FE00DA0975D84075A71075D80075D90475DA62
:10070E000975DB0975DC0975DD0975DE0975DF090B
:10071E0075D84075A70075E60875E71075BC0175AC
:10072E00BE0475BD6C75BE0775BDA075BE0875BDE2
:10073E000175BC0075BB1875BC2075BA0875E880CC
:10074E0075D11375B50075A70F75E10575E20075C6
:10075E00C740C293C294C291C292C287C290E5B5FD
:10076E0054EFF5B5E5B554DFF5B5C296C295C2A006
:10077E00C297C2A2C2A1E5B554BFF5B5E5B5547F87
:10078E00F5B5E5B554FBF5B5759700759780740A08
:10079E001252327597C0E5975420700280F8758F0B
:1007AE000275A700D2AF75980075A90C75A70F75C5
:1007BE00AB4375ADFB75AC1E75A71075C91875CA20
:1007CE000075CB0075C80475A700758912758E0467
:1007DE00758C00758A00C2A9D28C758D00758B0040
:1007EE00D2ABD28E75D944753200753100752E009C
:1007FE00752D00754600754700C29974C8F50975C8
:10080E00080012319675B50074639007B0F8E4F0E5
:10081E00E8A3F01234227464F509750800123196BB
:10082E00C21E90005AE0B40108A2B54002D21E804A
:10083E002E90005AE0B4021175A70F75F30F75A72D
:10084E0000A2A34002D21E801690005AE0B4030FFD
:10085E0075A70F75F31775A700A2A44002D21EA2AA
:10086E001EB3500302095B74089007B0F8E4F0E879
:10087E00A3F01232F17464F5097508001231967402
:10088E00099007B0F8E4F0E8A3F01232F17464F5C1
:10089E0009750800123196740A9007B0F8E4F0E872
:1008AE00A3F01232F17464F50975080012319674D2
:1008BE000B9007B0F8E4F0E8A3F01232F17464F58F
:1008CE0009750800123196740C9007B0F8E4F0E840
:1008DE00A3F01232F17464F50975080012319674A2
:1008EE000D9007B0F8E4F0E8A3F01232F17464F55D
:1008FE0009750800123196740E9007B0F8E4F0E80E
:10090E00A3F01232F17464F5097508001231967471
:10091E00029000B9F090005AE090007DF090005ADD
:10092E00E0B401087400900085F0801C90005AE03D
:10093E00B4020874009000C8F0800D90005AE0B424
:10094E00030674009000D5F0D21A020A3B9007B04D
:10095E00E4F0A304F01232F17464F5097508001284
:10096E00319674029007B0F8E4F0E8A3F01232F179
:10097E007464F50975080012319674039007B0F887
:10098E00E4F0E8A3F01232F17464F5097508001270
:10099E00319674049007B0F8E4F0E8A3F01232F147
:1009AE007464F50975080012319674059007B0F855
:1009BE00E4F0E8A3F01232F17464F5097508001240
:1009CE00319674069007B0F8E4F0E8A3F01232F115
:1009DE007464F50975080012319674079007B0F823
:1009EE00E4F0E8A3F01232F17464F5097508001210
:1009FE00319674019000B9F090005AE090007DF0AD
:100A0E0090005AE0B401087400900085F0801C90AC
:100A1E00005AE0B4020874009000C8F0800D9000F7
:100A2E005AE0B4030674009000D5F0C21A1235963F
:100A3E009000C3E07006740A9000C3F090006FE05F
:100A4E00700674E390006FF0120135E5B54401F5C0
:100A5E00B57406900049F0740190004AF07403904A
:100A6E00004CF0740490004DF0741590004EF0742C
:100A7E000590004FF090004BE0B404067404900013
:100A8E004FF07406900050F07400900055F0740012
:100A9E00900056F07401900057F07400900058F0DA
:100AAE0074FF900059F07433900147F07436900142
:100ABE0048F0742D900149F0743290014AF0742080
:100ACE0090014BF0743690014CF0744390014DF050
:100ADE00747990014EF0746C90014FF07420900177
:100AEE0050F07420900151F07420900152F0742057
:100AFE00900153F07420900154F07420900155F041
:100B0E009000DFE090006CF0900096E090006DF0A9
:100B1E00900097E090006EF0C213C215C21774C811
:100B2E00900028F074C890002CF074C8900030F03B
:100B3E00C210C211C212A2B6B39209A2B3B3920AE4
:100B4E00752600752500753746754C1E900068E4B5
:100B5E00F075271975286490000C74FFF0A374DCEF
:100B6E00F0C20D754B00C208752A00752900900061
:100B7E0010E4F0A3F0743A900770F074FD900771D2
:100B8E00F0756D00900069E4F0752C00752B0090E7
:100B9E000014E4F0A3F090009BE0900012F8E4F053
:100BAE00E8A3F090007CE075F032A4FFAEF0900068
:100BBE0022EEF0A3EFF09007AAE0FEA3E0FF74038D
:100BCE0012526074011252529007A8EEF0A3EFF089
:100BDE00754A01900045E4F0C222C21F756C007583
:100BEE003C00C20EC20FC223C203754D00C204D216
:100BFE0005C206D207C21BC21CD21D74FE90004055
:100C0E00F074FE900041F0C220D221753800754478
:100C1E0000753A00753E32753F00754000743C9089
:100C2E000043F0754100743C900044F0754200752D
:100C3E00430090001AE4F0A3F0754500D2B2D2A49E
:100C4E00D2B0D2B1D2A3D2A7D2A6D2A5D2B790009B
:100C5E007CE0D394FA400674FA90007CF07E017F1B
:100C6E000090006EE012526090006DE02FFF500178
:100C7E000E900024EEF0A3EFF0EFD394FFEE940F5E
:100C8E004007900024E4F0A3F090006CE07006742E
:100C9E00FF90006CF09000B9E0D39402400674010E
:100CAE009000B9F09000BAE07005754902800375A6
:100CBE0049039000BBE0D39401400674009000BB42
:100CCE00F09000C1E0C3940A5006740A9000C1F07F
:100CDE009000CBE0700674019000CBF09000CBE05A
:100CEE00B4FF0674FE9000CBF09000D2E0D394FED9
:100CFE00400674FE9000D2F074019000D8F074019A
:100D0E009000D9F074009000DBF074009000E0F0D9
:100D1E00D29CD2EC75CF01A298B35003021130C20F
:100D2E0098E54764046006E59964FF6002802AA294
:100D3E00204004D2208020E547600874E6254790C5
:100D4E000045F0754700E546600874F025469000B2
:100D5E0045F0754600C2208002C220E547600302BE
:100D6E000E0B754700E599B4FF03754601E599B47E
:100D7E00FE03754602E599B4FD03754603E599B485
:100D8E00FC03754604E599B4FA03754605E599B476
:100D9E00FB03754701E599B4F903754704E599D34B
:100DAE0094E54007E599C394F04002801685994872
:100DBE007547027E017F00E548C394E61252608EAD
:100DCE002F8F30753200753100E599D394C74007E7
:100DDE00E599C394E64002801F85994875470374D0
:100DEE00E5C39548F530752F00AE2FAF30904FD636
:100DFE00125221783112529BD299021130E547B42A
:100E0E0001028003020EE3AE31AF32900070125237
:100E1E0087E599F078311252BDAE31AF32EFB401A1
:100E2E0006EEB407028003020EE3900770E0B43CB6
:100E3E00028003020ECDC29C1205111201359000E4
:100E4E006CE09000DFF090006DE0900096F0900066
:100E5E006EE0900097F0A21A4032755001E550D323
:100E6E0094075026E5509007B0F8E4F0E8A3F0742C
:100E7E00AA90003DF01231C27464F5097508001293
:100E8E0031967850740126F650D38030755008E5AF
:100E9E0050D3940E5026E5509007B0F8E4F0E8A336
:100EAE00F074AA90003DF01231C27464F509750811
:100EBE00001231967850740126F650D3123596747E
:100ECE00C89007B0F8E4F0E8A3F0D29C754700751F
:100EDE0046007599FBE547B402028003020F8DE5CB
:100EEE00324531700685992E752D00AE31AF3274B4
:100EFE00016F4E701BAC2DAD2EAA2FAB30ED2BFB20
:100F0E00EC3AFA8A068B07900070125287E599F038
:100F1E0078311252BDAE31AF3274026F4E7060AC8A
:100F2E002DAD2E740D6D4C702C74639007B0F8E4DB
:100F3E00F0E8A3F074AB90003DF090007DE09000DF
:100F4E005AF01234FB90003DE4F074C89007B0F8EC
:100F5E00E4F0E8A3F0E548B4E619AE2DAF2E7456D2
:100F6E006F4E600C74486F4E600674666F4E700361
:100F7E00120511120135854899754700754600E531
:100F8E0047B4033FAE31AF32900070125287E599ED
:100F9E00F078311252BDAE31AF32AC2FAD308F0280
:100FAE008E038C068D07905012125221E493F97421
:100FBE000193FEEAD39EEB99400985489975470047
:100FCE00754600E547B404028003021130AE31AF1E
:100FDE0032900070125287E599F078311252BDAE00
:100FEE0031AF32EFB40006EEB401028003021130CD
:100FFE00120511900053E075F002A4FFAEF08F5071
:10100E00EF900070125292EFFCE0FDEC9000731224
:10101E005292EDFCE0FDEC2DFC900053E0B5040285
:10102E0080030211210FEF900070125292E550FFD3
:10103E00E0FCEF900074125292ECFFE0FCEFC39CC8
:10104E00FF900053E0B507028003021121E5509096
:10105E000072125292E550FFE0FCEF9000751252B2
:10106E0092ECFFE0FCEF2CFF900053E0B5070280FE
:10107E0003021121E550900076125292FFE0FCEF30
:10108E00900053E0F4042C90005AF0E55090007755
:10109E00125292FFE0FCEF900053E0F4042C90000B
:1010AE005BF0E550900078125292FFE0FCEF90005A
:1010BE0053E0F4042C90005CF0E55090007912524D
:1010CE0092FFE0FCEF900053E0F4042C9007B0F890
:1010DE00E4F0E8A3F074AB90003DF01234FB7464BE
:1010EE00F5097508001231969007B012526E12343F
:1010FE00FB7464F5097508001231969007B0125210
:10110E006E1234FB7599F97464F509750800123185
:10111E009680FE7599FF7464F50975080012319674
:10112E0080FEE5466006A299B3B340030212B0C238
:10113E0099E546B4011FAE31AF3290004912528785
:10114E00E0F59978311252BDAE31AF3274116F4E57
:10115E007003754600E546B40203854A99E546B428
:10116E00031DAE31AF32900070125287E0F599EF49
:10117E00B40107EEB4070375460078311252BDE58F
:10118E0046B404028003021272E5324531700385C3
:10119E002699AE31AF3274016F4E7003853899AE19
:1011AE0031AF3274026F4E7003853A99AE31AF3261
:1011BE0074036F4E7003853E99AE31AF3274046F77
:1011CE004E7003854099AE31AF3274056F4E700389
:1011DE00854199AE31AF3274066F4E7003854299D8
:1011EE00AE31AF3274076F4E7003854399AE31AF97
:1011FE003274086F4E700690001BE0F599AE31AF59
:10120E003274096F4E7017A221B340077599FAC256
:10121E0021800B900045E0F599900045E4F0AE3149
:10122E00AF32740A6F4E7003854499AE31AF32748B
:10123E000B6F4E7003853F99AE31AF32740C6F4E0B
:10124E007003854599AE31AF32740D6F4E700375D4
:10125E0099FC78311252BDAE31AF32740E6F4E70B2
:10126E0003754600E546B4053990004BE0D394046F
:10127E004010AE31AF32904D8A125287E493F599F9
:10128E00800EAE31AF32904E6E125287E493F599C6
:10129E00AE31AF3274E36F4E700375460078311283
:1012AE0052BDE54764016005E547B40403020D2213
:1012BE00C28E7E107F00E53D125260E58D75F010F6
:1012CE00A4FDACF0EF2DFDEE3CFCE58B75F010842B
:1012DE00FF7E00ED2FFFEC3EFE8E278F28D28E90E4
:1012EE00009DE0605690001C12526E90001CE0FCB7
:1012FE00A3E0FD90001EE0FAA3E0FBEDB5033CEC8D
:10130E00B50238B219A208B34013A219B34008E5CA
:10131E00B54404F5B58006E5B554FBF5B590001E51
:10132E00E0FEA3E0FF900020E0FCA3E0FDEF2DFD2A
:10133E00EE3CFC90001EECF0A3EDF09000AAE060F5
:10134E00099000AAE0C394034003021411124AD07C
:10135E00A208B35009900068E0C3942840028006AA
:10136E00900094E0F56BE56B75F005A4FFAEF09080
:10137E0007B2EEF0A3EFF0900081E0C3953A40077C
:10138E00E538C3953950079007B2E4F0A3F0AE5894
:10139E00AF599007B2E0FCA3E0FDEFD39DEE9C4069
:1013AE0022C2A1E5B554DFF5B59000AAE0B402095A
:1013BE009000B8E0C3940340028006E5B54410F5F2
:1013CE00B58029900068E0C3943C5002D2A1E5B5E7
:1013DE004420F5B59000AAE0B402099000B8E0C32D
:1013EE00940340028006E5B554EFF5B59000AAE0EF
:1013FE00B402099000B8E0C3940340028005A2A194
:10140E00B392A29000AAE0B4031C124BEBAE58AFFD
:10141E00599007B2E0FCA3E0FDEFD39DEE9C400493
:10142E00D2A18002C2A1900085E06009A2B3300A69
:10143E0001B3B340028039A2B3300A01B34031A2E6
:10144E00B3300C01B3401C9000B8E0B40306A21BED
:10145E00B3B3400280067405900045F0D21BA20C77
:10146E00B3920AA20CB330B301B34004A20C920A99
:10147E00A2B6300901B35003021A45A2B6300901D3
:10148E00B35003021A45A2B6300B01B35003021932
:10149E005C754A0090009DE07013A20BB34008E506
:1014AE00B554FBF5B58006E5B54404F5B50537A290
:1014BE000DB3B35013AE27AF2890000CE0FCA3E0A1
:1014CE00FDEDC39FEC9E40030215D3E549B40330F6
:1014DE00E537B42305754901801FA222B3401AE5F2
:1014EE0037C3942350069000457401F0E537D3942A
:1014FE002340067402900045F0753701D222805CBD
:10150E00E549B40206754901753723E537B423055D
:10151E007537018047900045E07032E537C394235C
:10152E0050069000457401F0E537D39423400674BD
:10153E0002900045F0E537C394235002D21FE537E1
:10154E00D394234002D21FC296C295C2A09000BA75
:10155E00E0B402051205118003753701AE29AF2ADA
:10156E00AC27AD28EF2DFDEE3CFC74028C068D07EA
:10157E001252528E298F2A90009DE0603F90001CDF
:10158E00E0FCA3E0FD90009DE0FF12524274018C3E
:10159E00068D07125252900020EEF0A3EFF090004D
:1015AE0020E0F8A3E090001EC8F0A3C8F090001C45
:1015BE00E4F0A3F0C219E5B554FBF5B5A21FB34094
:1015CE0002C21F802BAE29AF2AAC27AD28EF2DFD0E
:1015DE00EE3CFC74018C068D071252528E298F2A16
:1015EE00AC27AD28EDD39488EC941340031205116B
:1015FE00E537B423127403900045F0D21F9000BA61
:10160E00E0B40203120511AE2BAF2CAC27AD28EFC0
:10161E002DFDEE3CFC8C2B8D2CAE27AF28EFD39DF1
:10162E00EE9C4011900014E0FAA3E0FBEBC394E8AB
:10163E00EA94034002800690001412526E9000103D
:10164E00E0FEA3E0FFAC27AD28EF2DFDEE3CFC90B5
:10165E000010ECF0A3EDF09000BAE0B40218AE2743
:10166E00AF287405125260740112525290000CEEA3
:10167E00F0A3EFF08011AE27AF28740212526090E3
:10168E00000CEEF0A3EFF0C28E758D00758B007519
:10169E003D00752801752700D28EE537240875F0B8
:1016AE000984AFF07E00EF4E7075900010E0F8A345
:1016BE00E090000EC8F0A3C8F090000EE0FEA3E08C
:1016CE00FFEF4E600B7C807D0E1251408E258F26D3
:1016DE00900010E4F0A3F0AE25AF267428BE0003F0
:1016EE009F5010E53C2FFF50010E74011252528E86
:1016FE00258F2685263C9000C1E0A825B8000DD385
:10170E0095264008E526900042F080099000C1E041
:10171E0014900042F0E5496006752600752500908C
:10172E0000B8E0B40308900037E065376002802609
:10173E00A21BB34004D21C8002B21C900085E06054
:10174E000BA21BB35006A21CB3B340028006740456
:10175E00900045F0C21BE537640B6005E537B41DFC
:10176E00099000AAE060031247D89000AFE0B401E0
:10177E001490003EE06537600790003FE0B53703F8
:10178E00754B00801E90003EE06537601390003E62
:10179E00E0240C6537600990003EE02418B537034D
:1017AE00754B00A20EB35006A20DB3B34003021840
:1017BE00B1900076E0B4015AE54075F00584FF7EE5
:1017CE0000900570125287E0F534753300AE33AFDA
:1017DE0034900074E012526074648E048F05FF1210
:1017EE00524274C18C068D071252608E358F369020
:1017FE000012E0FEA3E0FFAC33AD341200037464BC
:10180E008E048F05FF125242900012ECF0A3EDF001
:10181E00800F900074E075F0C1A4FFAEF08E358F8E
:10182E0036E53AC394CC5006900074E07002807195
:10183E0075A71085F95085FA517E017F00E551128A
:10184E005260E5502FFF50010E8E338F34AC35AD04
:10185E0036EF2DFDEE3CFC8C358D36D293D294D2E4
:10186E0091E536F5FBE535F5FCE536F5E9E535F5BB
:10187E00EAE536F5EBE535F5EC9000B8E0B4031E7D
:10188E00D292D287D290E536F5EDE535F5EEE53616
:10189E00F5FDE535F5FEE536F5CEE535F5CF75A763
:1018AE0000D20EE549B40106E537640B6002800FE5
:1018BE00754C019000487401F0E5B54401F5B5E5AD
:1018CE004960030219579000BDE0600D9000C4E01E
:1018DE00A825B8000695264002803A9000BDE0B4D7
:1018EE00021F900034E06537600F900035E06537D9
:1018FE006007900036E0B53703754C0375450080E0
:10190E000CC20075450090001AE4F0A3F074099023
:10191E000045F08034900034E0B5370B754C0190E3
:10192E0000487401F08022900035E0B5370B754CFD
:10193E00017402900048F08010900036E0B537092F
:10194E00754C017403900048F0A20BB39209A20BE0
:10195E00B330B601B35003021A45754A0190009D8B
:10196E00E07013A20BB34008E5B54404F5B580064C
:10197E00E5B554FBF5B5A20B9209E537D3944A4071
:10198E0014D20DE537D3946D400B7403900045F0DF
:10199E00D21F7537469000C5E0B40107E543C394E6
:1019AE0014400280031205117428900068F0A204FE
:1019BE00300501B35017A204B34008E5B54408F54D
:1019CE00B58006E5B554F7F5B5A2049205A206302A
:1019DE000701B35017A206B34008E5B54402F5B5AA
:1019EE008006E5B554FDF5B5A2069207E543C3940E
:1019FE00415009740E900045F012051190004FE011
:101A0E00FE90004BE004C39E400990004BE0D3943F
:101A1E0006400974FB900045F0120511900054E049
:101A2E006015900054E0FE90004EE06E600974FE6A
:101A3E00900045F0120511A21FB34006C296C29542
:101A4E00C2A0A210B3B35008900037E06537600310
:101A5E00021B3EA202B35006A200B3B34003021B08
:101A6E003875A71085F95085FA517E017F00E55132
:101A7E00125260E5502FFF50010E8E338F349000BE
:101A8E0018E0FCA3E0FDEF2DFDEE3CFC8C358D3611
:101A9E009000B8E0B4034EA208B34028A21CB34095
:101AAE000CE536F5FBE535F5FCD293800AE536F507
:101ABE00EDE535F5EED292A203B34004D2A2800238
:101ACE00C2A2801FE536F5FBE535F5FCE536F5EDF2
:101ADE00E535F5EED293D292A203B34004D2A280A2
:101AEE0002C2A280429000D6E0C394025013E536A3
:101AFE00F5FBE535F5FCD293A203B34002D29280FA
:101B0E0026E536F5FBE535F5FCD293AE33AF34ACB6
:101B1E0056AD57EF2DFDEE3CFC8C358D36E536F58A
:101B2E00EDE535F5EED29275A700C210D211D212A4
:101B3E00A211B3B35008900038E065376003021C61
:101B4E002CA202B35006A200B3B34003021C2675AA
:101B5E00A71085F95085FA517E017F00E55112528A
:101B6E0060E5502FFF50010E8E338F34900018E039
:101B7E00FCA3E0FDEF2DFDEE3CFC8C358D36900088
:101B8E00B8E0B4034EA208B34028A21CB3400CE543
:101B9E0036F5E9E535F5EAD294800AE536F5FDE548
:101BAE0035F5FED287A203B34004D2A28002C2A2B0
:101BBE00801FE536F5E9E535F5EAE536F5FDE5355F
:101BCE00F5FED294D287A203B34004D2A28002C201
:101BDE00A280429000D6E0C394025013E536F5E998
:101BEE00E535F5EAD294A203B34002D2878026E50A
:101BFE0036F5E9E535F5EAD294AE33AF34AC56ADF1
:101C0E0057EF2DFDEE3CFC8C358D36E536F5FDE5BA
:101C1E0035F5FED28775A700D210C211D212A212CC
:101C2E00B3B35008900039E065376003021D1AA265
:101C3E0002B35006A200B3B34003021D1475A710E1
:101C4E0085F95085FA517E017F00E551125260E50B
:101C5E00502FFF50010E8E338F34900018E0FCA3EE
:101C6E00E0FDEF2DFDEE3CFC8C358D369000B8E09E
:101C7E00B4034EA208B34028A21CB3400CE536F5BF
:101C8E00EBE535F5ECD291800AE536F5CEE535F586
:101C9E00CFD290A203B34004D2A28002C2A2801F70
:101CAE00E536F5EBE535F5ECE536F5CEE535F5CF74
:101CBE00D291D290A203B34004D2A28002C2A280DB
:101CCE00429000D6E0C394025013E536F5EBE535AD
:101CDE00F5ECD291A203B34002D2908026E536F500
:101CEE00EBE535F5ECD291AE33AF34AC56AD57EFE4
:101CFE002DFDEE3CFC8C358D36E536F5CEE535F515
:101D0E00CFD29075A700D210D211C212E54CB408F2
:101D1E0018124107A210B35005A211B3400280065B
:101D2E00D210D211D212754C1EE54CB40706123EDB
:101D3E00BF754C08E54CB4063D900012E0FEA3E0E2
:101D4E00FFEF4E6006A208B3B340028023AE52AF3F
:101D5E0053900012E0FCA3E0FDEF2DFDEE3CFC8C59
:101D6E00528D53E537D3940C500690001212003961
:101D7E00123C91754C07E54CB40506123AF1754CC0
:101D8E0006E54CB404329000ABE0903178F8282888
:101D9E00731237858012123785800D123933800801
:081DAE001239E580031239E54A
:0F317800021D9F021DA4021DA9021DAE021DB360
:101DB60090008DE060051248C18002C204754C0592
:101DC600E54CB403028003021EB0900090E060056B
:101DD6001249CE8002C2069000ABE0D39402403F87
:101DE60090007FE02403A825B800049526500990AA
:101DF6000081E0D3953A50028008D2027408900020
:101E060045F090007FE0A825B80005D39526500B35
:101E1600900081E02403C3953A5002C202803990B3
:101E2600007FE02403A825B8000495265007E5386E
:101E3600C3953940028008D2027408900045F0909C
:101E4600007FE0A825B80005D395265009E539247A
:101E56000FC395385002C2029000C5E07007E543F3
:101E6600C3941440028002D202A2024005754C04BB
:101E7600800A754C1E90001AE4F0A3F0A208B34045
:101E860029E54075F00584FF7E00900570125287A3
:101E9600E0C39469500512480D800F9007AAE0F838
:101EA600A3E09007A8C8F0A3C8F0E54CB40A0280E6
:101EB60003021F7290002AE0C394465008C296742B
:101EC6004690002AF090003AE0B4011DE55A240A33
:101ED600F55A9007ACE0FEA3E0FF740A2FFF50010D
:101EE6000E9007ACEEF0A3EFF090003AE0B4021DBE
:101EF600E55A2414F55A9007ACE0FEA3E0FF7414EB
:101F06002FFF50010E9007ACEEF0A3EFF0855A3488
:101F1600753300900034E0F55012009EE5369000CF
:101F26002AF0900006E533F0A3E534F0E550900082
:101F36002BF0C2149007ACE0F533A3E0F534900023
:101F460034E0F55012009EE536900028F09000002F
:101F5600E533F0A3E534F0E550900029F0C213E52F
:101F660049B40105754C0B8003754C03900028E0BD
:101F7600B537028003022014A2134072900000E0DD
:101F8600FEA3E0FFEF4E6021AE29AF2A900000E0ED
:101F9600FCA3E0FD120003740A8E048F05FF1252A3
:101FA60042900000ECF0A3EDF0900029E0601A905A
:101FB6000000E0FEA3E0FFAC29AD2AEF2DFDEE3CCC
:101FC600FC900000ECF0A3EDF0900029E0D3940122
:101FD600401A900000E0FEA3E0FFAC29AD2AEF2DE9
:101FE600FDEE3CFC900000ECF0A3EDF0D213AE2722
:101FF600AF28900000E0FCA3E0FDEFC39DEE9C40FF
:102006000D1205DBD296C21374C8900028F0A213F5
:10201600B3B35007900028E0B53702800D1205DBF8
:10202600D29674C8900028F0C21390002AE0B53703
:102036000280030220CFA2144072900006E0FEA3A5
:10204600E0FFEF4E6021AE29AF2A900006E0FCA328
:10205600E0FD120003740A8E048F05FF12524290AF
:102066000006ECF0A3EDF090002BE0601A9000065D
:10207600E0FEA3E0FFAC29AD2AEF2DFDEE3CFC907F
:102086000006ECF0A3EDF090002BE0D39401401A8B
:10209600900006E0FEA3E0FFAC29AD2AEF2DFDEE91
:1020A6003CFC900006ECF0A3EDF0D214AE27AF286E
:1020B600900006E0FCA3E0FDEFC39DEE9C400AC243
:1020C60096744690002AF0C214A214B3B350079037
:1020D600002AE0B53702800AC296744690002AF0BC
:1020E600C214E54CB40B0280030221B590002EE029
:1020F600C3944650139000C6E0B40104C296800211
:10210600C295744690002EF090003BE0B4011DE5A8
:102116005A240AF55A9007ACE0FEA3E0FF740A2F92
:10212600FF50010E9007ACEEF0A3EFF090003BE0FD
:10213600B4021DE55A2414F55A9007ACE0FEA3E05C
:10214600FF74142FFF50010E9007ACEEF0A3EFF0D2
:10215600855A34753300900035E0F55012009EE53F
:102166003690002EF0900008E533F0A3E534F0E554
:102176005090002FF0C2169007ACE0F533A3E0F5BF
:1021860034900035E0F55012009EE53690002CF0B4
:10219600900002E533F0A3E534F0E55090002DF011
:1021A600C215E549B40105754C0C8003754C0390C6
:1021B600002CE0B537028003022262A2154072901D
:1021C6000002E0FEA3E0FFEF4E6021AE29AF2A90A9
:1021D6000002E0FCA3E0FD120003740A8E048F05E2
:1021E600FF125242900002ECF0A3EDF090002DE0B9
:1021F600601A900002E0FEA3E0FFAC29AD2AEF2DA5
:10220600FDEE3CFC900002ECF0A3EDF090002DE01A
:10221600D39401401A900002E0FEA3E0FFAC29AD82
:102226002AEF2DFDEE3CFC900002ECF0A3EDF0D27F
:1022360015AE27AF28900002E0FCA3E0FDEFC39D9A
:10224600EE9C40181205DB9000C6E0B40104D2965D
:102256008002D295C21574C890002CF0A215B3B3B3
:10226600500790002CE0B5370280181205DB90006D
:10227600C6E0B40104D2968002D29574C890002CB0
:10228600F0C21590002EE0B537028003022333A278
:10229600164072900008E0FEA3E0FFEF4E6021AE0C
:1022A60029AF2A900008E0FCA3E0FD120003740A9F
:1022B6008E048F05FF125242900008ECF0A3EDF059
:1022C60090002FE0601A900008E0FEA3E0FFAC2922
:1022D600AD2AEF2DFDEE3CFC900008ECF0A3EDF0EE
:1022E60090002FE0D39401401A900008E0FEA3E08E
:1022F600FFAC29AD2AEF2DFDEE3CFC900008ECF07A
:10230600A3EDF0D216AE27AF28900008E0FCA3E0BC
:10231600FDEFC39DEE9C40159000C6E0B40104C2DB
:10232600968002C295744690002EF0C216A216B38D
:10233600B3500790002EE0B5370280159000C6E036
:10234600B40104C2968002C295744690002EF0C273
:1023560016E54CB40C028003022422900032E0C33E
:10236600944650139000C6E0B40104C2968002C29F
:10237600A07446900032F090003CE0B4011DE55A8E
:10238600240AF55A9007ACE0FEA3E0FF740A2FFF7B
:1023960050010E9007ACEEF0A3EFF090003CE0B4D5
:1023A600021DE55A2414F55A9007ACE0FEA3E0FF9F
:1023B60074142FFF50010E9007ACEEF0A3EFF085DA
:1023C6005A34753300900036E0F55012009EE5361B
:1023D600900032F090000AE533F0A3E534F0E550C2
:1023E600900033F0C2189007ACE0F533A3E0F53463
:1023F600900036E0F55012009EE536900030F090E1
:102406000004E533F0A3E534F0E550900031F0C266
:1024160017E549B40103754900754C03900030E097
:10242600B5370280030224CFA2174072900004E061
:10243600FEA3E0FFEF4E6021AE29AF2A900004E034
:10244600FCA3E0FD120003740A8E048F05FF1252EE
:1024560042900004ECF0A3EDF0900031E0601A9099
:102466000004E0FEA3E0FFAC29AD2AEF2DFDEE3C13
:10247600FC900004ECF0A3EDF0900031E0D3940161
:10248600401A900004E0FEA3E0FFAC29AD2AEF2D30
:10249600FDEE3CFC900004ECF0A3EDF0D217AE2765
:1024A600AF28900004E0FCA3E0FDEFC39DEE9C4046
:1024B600181205DB9000C6E0B40104D2968002D261
:1024C600A0C21774C8900030F0A217B3B35007909B
:1024D6000030E0B5370280181205DB9000C6E0B484
:1024E6000104D2968002D2A074C8900030F0C217C0
:1024F600900032E0B5370280030225A0A218407290
:1025060090000AE0FEA3E0FFEF4E6021AE29AF2A5D
:1025160090000AE0FCA3E0FD120003740A8E048F0B
:1025260005FF12524290000AECF0A3EDF090003342
:10253600E0601A90000AE0FEA3E0FFAC29AD2AEFA6
:102546002DFDEE3CFC90000AECF0A3EDF09000337C
:10255600E0D39401401A90000AE0FEA3E0FFAC2904
:10256600AD2AEF2DFDEE3CFC90000AECF0A3EDF059
:10257600D218AE27AF2890000AE0FCA3E0FDEFC317
:102586009DEE9C40159000C6E0B40104C296800200
:10259600C2A07446900032F0C218A218B3B3500716
:1025A600900032E0B5370280159000C6E0B4010411
:1025B600C2968002C2A07446900032F0C218E54C62
:1025C600B4020280030226741245701246879007F1
:1025D600A8E0FEA3E0FF740A12526090000EE0FC31
:1025E600A3E0FD74098F02FF1252428D078C038E01
:1025F600048A058B061251409007ACEEF0A3EFF06B
:102606009000C6E0B401087450BE00059F400280E9
:102616000D74509007ACF8E4F0E8A3F0801B900727
:10262600ACE0FEA3E0FF74F0BE00039F500B74F015
:102636009007ACF8E4F0E8A3F09007ACE0FEA3E066
:10264600FFE55A2FFF50010E9007ACEEF0A3EFF016
:10265600900048E0B40103754C0A900048E0B402CB
:1026660003754C0B900048E0B40303754C0CE54C25
:10267600B401259000DDE0903187F82828731243D5
:102686000E801212430E800D1243988008124444A5
:05269600800312444422
:0F31870002268402268902268E022693022698AB
:10269B00754C029000C8E0B4020280030227B6908A
:1026AB00006BE0D3953F506490006BE0F404253F42
:1026BB00FE9000CBE08E00F5F0E884FF7E008F509B
:1026CB00EFC39410500CEF8550F0A4FDACF08D507F
:1026DB0080037550FF90006BE0D39550400B90003A
:1026EB006BE0C39550F54D8003754D009000E6E00F
:1026FB00D3954D40069000E6E0F54D9000E7E0C322
:10270B00954D50069000E7E0F54D807190006BE021
:10271B00C3953FFE9000CBE08E00F5F0E884FF7E82
:10272B00008F50EFC39410500CEF8550F0A4FDAC0C
:10273B00F08D5080037550FF855034753300900039
:10274B006BE02534FFAE3350010E8E338F3474FFA4
:10275B00BE0009D39F400585344D8003754DFF9016
:10276B0000E6E0D3954D40069000E6E0F54D900075
:10277B00E7E0C3954D50069000E7E0F54DA208B396
:10278B00B350099000D3E0D3954E5002800A7407E2
:10279B00900045F0C297801375A710E5CDC3954DFA
:1027AB004004C2978002D29775A700E54BC39409EA
:1027BB004003022EF1A2EDB35003022EF1C2EDE560
:1027CB004B6003022965900079E070030229549055
:1027DB0000AFE0B4010280030228B490003EE0B5E4
:1027EB00370280030228B17E017F00E5BE125260E2
:1027FB00E5BD2FFF50010E8E338F34900079E0B47E
:10280B000118741012526090006FE08E048F05FF58
:10281B00125242ED900040F0802CAE33AF34741066
:10282B0012526090006FE08E048F05FF125242909F
:10283B000040E02DFD50010C74018C068D071252E7
:10284B0052EF900040F0E54460089000D5E0640240
:10285B00600280219000D7E0B4011A900040E0752F
:10286B00F0E7A4FFAEF0E5448E048F05FF12524251
:10287B00ED900040F0900040E0FE900041E0D39ED0
:10288B004004D21D8002B21D900040E0900041F048
:10289B009000ABE064016006A21DB3B3400280065A
:1028AB00900040E0F538022952D21D7E017F00E5F1
:1028BB00BE125260E5BD2FFF50010E8E338F349048
:1028CB000079E0B40118741012526090006FE08E22
:1028DB00048F05FF125242ED900040F0802CAE3376
:1028EB00AF34741012526090006FE08E048F05FFAE
:1028FB00125242900040E02DFD50010C74018C06E9
:10290B008D07125252EF900040F0E54460089000A2
:10291B00D5E06402600280219000D7E0B4011A90E8
:10292B000040E075F0E7A4FFAEF0E5448E048F05A0
:10293B00FF125242ED900040F09000ABE06401605A
:10294B0006900040E0F5388003753800900075E084
:10295B007005754B01800375BB18E54BB401028004
:10296B0003022B07900075E07003022AF67E017FAD
:10297B0000E5BE125260E5BD2FFF50010E8E338F66
:10298B00349000BBE0B4010F7E0F7FFFAC33AD344E
:10299B001252B58E338F349000E0E0B40245AE3363
:1029AB00AF34900024E0FCA3E0FDEDD39FEC9E4000
:1029BB000A900024E533F0A3E534F0AE33AF349046
:1029CB000026E0FCA3E0FDEFD39DEE9C400A9000B7
:1029DB0026E533F0A3E534F0AE33AF347404125272
:1029EB00528F3A9000E0E0704CAE33AF349000243D
:1029FB00E0FCA3E0FDEFD39DEE9C40091252B58E97
:102A0B00338F348006753400753300AE33AF3474B6
:102A1B001012526090006CE08E048F05FF12524230
:102A2B008C338D347400D39D74019C400585343AEE
:102A3B008003753AFF9000ABE0B401028003022AD9
:102A4B00F4A208B3B3500E90007FE0A825B80005A0
:102A5B00D395265003022AE9900080E075F019A463
:102A6B00FFAEF09000C3E08E048F05FF1252429030
:102A7B0000BCE0853AF0A4FFAEF074648D028C03C9
:102A8B008E048F05FF125242EA2DFDEB3CFC8C337A
:102A9B008D34E544600F9000D5E0B402089000D768
:102AAB00E0640160028017AE33AF3474E7125260FA
:102ABB00E5448E048F05FF1252428C338D34900007
:102ACB0040E0A833B8000AD39534400585343880EC
:102ADB000BA21DB34006900040E0F538800BA21D01
:102AEB00B34006900040E0F5388003753A00900043
:102AFB0078E07005754B02800375BB19E54BB4028A
:102B0B00028003022BC2900078E07003022BB1E528
:102B1B0037D3940C4003022BAF900022E0FEA3E0CE
:102B2B00FFE53E1252AD900022EEF0A3EFF07E01D6
:102B3B007F00E5BE125260E5BD2FFF50010E8E33B4
:102B4B008F349000E5E07013740A12526074518E4A
:102B5B00048F05FF1252428D3E8019AE33AF347491
:102B6B000A1252608F048E057E017F95CDCCCD125B
:102B7B0051408F3EE53ED394644003753E64900014
:102B8B0022E0FEA3E0FFE53E2FFF50010E90002256
:102B9B00EEF0A3EFF090007CE0048E048F05FF12A3
:102BAB0052428D3E8003753E329000C8E070057531
:102BBB004B03800375BB13E54BB4035E9000C8E079
:102BCB0060477E017F00E5BE125260E5BD2FFF50CE
:102BDB00010E8E338F3474041252528F3F9000CA01
:102BEB00E0853FF0A4FDACF07464FF1252428D3FC0
:102BFB009000C9E0853FF0A4FFAEF074FF8E048F08
:102C0B0005FF1252428D4E8003753F00900076E017
:102C1B007005754B04800375BB17E54BB40402803C
:102C2B0003022CC3900076E0B4017C7E017F00E5AB
:102C3B00BE125260E5BD2FFF50010E7404125252AA
:102C4B008E338F34900043E06012900043E0149079
:102C5B00504E93A833B8000695344002800690007E
:102C6B0043E014F0900043E0C3947750139000437B
:102C7B00E00490504E93A833B80005D3953450021E
:102C8B008006900043E004F0900043E0FE90009C2F
:102C9B00E08E0088F0A4FFAEF074648E048F05FF05
:102CAB001252428D408003754000900077E0700512
:102CBB00754B05800375BB16E54BB405028003020B
:102CCB002D56900077E0B4017C7E017F00E5BE12AB
:102CDB005260E5BD2FFF50010E74041252528E3319
:102CEB008F34900044E06012900044E0149050C781
:102CFB0093A833B80006953440028006900044E058
:102D0B0014F0900044E0C394775013900044E00417
:102D1B009050C793A833B80005D395345002800662
:102D2B00900044E004F0900044E0FE9000A2E08E9E
:102D3B000088F0A4FFAEF074648E048F05FF12526E
:102D4B00428D41800375410075BB1FE54BB40633C3
:102D5B007E017F00E5BE125260E5BD2FFF50010ED4
:102D6B008E338F34740912526074E68E048F05FF14
:102D7B001252428D4390007EE07005754B07800325
:102D8B0075BB15E54BB407028003022E9890007EAD
:102D9B00E07003022E877E017F00E5BE125260E5D4
:102DAB00BD2FFF50010E8E338F3474041252528F8D
:102DBB004290007EE0B401159000D2E08542F0A471
:102DCB00FFAEF07407125252EF9007B5F090007EF1
:102DDB00E0B402159000D2E08542F0A4FFAEF0748F
:102DEB0007125252EF9007B4F090007EE0B403024A
:102DFB008003022E859000BFE0701CE542C3940A4D
:102E0B005002D201E542D394644002C20190009E6D
:102E1B00E090006AF0806390009EE070349000D2E6
:102E2B00E08542F0A4FFAEF074FF8E048F05FF1215
:102E3B005242ED90006AF0AE25AF26741EBE00061E
:102E4B00D39F4002D201E53AD394E54002C2018000
:102E5B0029E542C3940A500DAE25AF26741EBE0061
:102E6B0004D39F50028002D201E53AD394E540028D
:102E7B00C20190009EE090006AF0800375420090C2
:102E8B0000D5E07005754B08800375BB14E54BB49A
:102E9B0008509000D5E060397E017F00E5BE1252EC
:102EAB0060E5BD2FFF50010E8E338F34EFD394218D
:102EBB00EE940E40057544FF8015AE33AF3474109D
:102ECB0012526074E38E048F05FF1252428D4480C0
:102EDB0003754400900079E0600575BB1A8003759B
:102EEB00BB18054BD2ECAE27AF287428C39F7423B5
:102EFB009E400C900069E0C3943C4003023175C2C4
:102F0B000D7537469000BAE0700575490280037560
:102F1B004903C293C294C291C292C287C290E5B5D3
:102F2B0054EFF5B5E5B554DFF5B5C296C295C2A021
:102F3B00C297C2A2C2A1E5B554BFF5B5E5B5547FA2
:102F4B00F5B5A21EB34008E5B54404F5B58006E51A
:102F5B00B554FBF5B5A20FB3500EE53AD3943340FD
:102F6B0007E53AC394CC4003023013E5B54401F5B1
:102F7B00B57428900068F0900074E075F064A4FFBD
:102F8B00AEF08E358F367402BE000AD39F400675A5
:102F9B00360275350075A71085F95085FA517E01FB
:102FAB007F00E551125260E5502FFF50010E8E331A
:102FBB008F34AC35AD36EF2DFDEE3CFC8C358D36BC
:102FCB00D293D294D291E536F5FBE535F5FCE53697
:102FDB00F5E9E535F5EAE536F5EBE535F5EC900089
:102FEB00B8E0B4031ED292D287D290E536F5EDE568
:102FFB0035F5EEE536F5FDE535F5FEE536F5CEE5D1
:10300B0035F5CF75A700D20FE53AC3941A5002C21B
:10301B000F90000C74FFF0A374DCF090009BE09019
:10302B000012F8E4F0E8A3F0C213C215C21774C87B
:10303B00900028F074C890002CF074C8900030F009
:10304B00C210C211C212752600752500753C00C254
:10305B0008756C0090001AE4F0A3F0754C1E9007F5
:10306B00AAE0FEA3E0FF74031252607401125252E5
:10307B009007A8EEF0A3EFF090008DE060051248EA
:10308B00C18002C204900090E060051249CE80021C
:10309B00C206A204300501B35017A204B34008E5E1
:1030AB00B54408F5B58006E5B554F7F5B5A204921D
:1030BB0005A206300701B35017A206B34008E5B5C9
:1030CB004402F5B58006E5B554FDF5B5A2069207A9
:1030DB00C203752C00752B00900014E4F0A3F09044
:1030EB00007CE075F032A4FFAEF0900022EEF0A36E
:1030FB00EFF0900010E4F0A3F0C222900069E0C35F
:10310B00943C5010E54BB40909900069E004F0754C
:10311B004B00803BE54BB40903754B0075280075DC
:10312B002700758D00758B00753D00900068E0C31E
:10313B00943C5008900068E004F08006743C9000CA
:10314B0068F0900068E0B43C06E5B554FEF5B59028
:10315B000069E0D394014007E543C39441400280EA
:0D316B0009740E900045F0120511020D22AE
:104FD6000000010001400160018001A001C001E064
:104FE60002000300039603B603D603F4040005008B
:104FF60005180530054805600578059005A805C023
:10500600060006140628063C066E068C00FF013FC5
:10501600015F017F019F01BF01DF01FF02FF0395D1
:1050260003B503D503F303FF04FF0517052F054753
:10503600055F0577058F05A705BF05FF061306273C
:10504600063B066F068B06A9DAD8D7D5D4D2D0CFC1
:10505600CDCBC9C7C6C4C2C0BEBCBAB8B5B3B1AF62
:10506600ADABA8A6A4A2A09D9B99969492908D8B79
:1050760089878482807E7C79777573716F6D6B69A1
:10508600676563615F5D5B5957565452504F4D4B90
:105096004A4847454442413F3E3C3B3A393736351C
:1050A600343231302F2E2D2C2B2A29282726252540
:1050B6002423222121201F1E1E1D1C1C1B1A1A1907
:1050C60019EEECEBEAE9E8E7E5E4E3E1E0DEDDDB57
:1050D600D9D8D6D4D2D0CECCCAC8C6C3C1BFBCBA22
:1050E600B7B5B2B0ADABA8A5A3A09D9B989592907D
:1050F6008D8A8785827F7D7A7775726F6D6A68651E
:1051060063615E5C5A575553514F4D4B4947454372
:1051160042403E3C3B393836353332312F2E2D2B2B
:105126002A292827262524232221201F1E1D1D1C4F
:0A5136001B1A1A191818171616157F
:10319600750B00750A00AE0AAF0BAC08AD09EDC39E
:1031A6009FEC9E401674FF12523275CF01780B7455
:1031B6000126F6500418E436F650DB2290003DE076
:1031C600B4AA1C900770E0B43C159007B0E0FEA3CB
:1031D600E0FFEF4E6009741EBE0004D39F50030249
:1031E60032F075360075350075F8099007B0E0FEC7
:1031F600A3E0FF74076F4E6006740E6F4E70067480
:103206003A900770F09007B0E0FEA3E0FF7408BEA6
:10321600001ED39F401A7E017F089007B0E0FCA3F2
:10322600E0FD1DBDFF011C1200038E338F34801F8D
:103236009007B0E0FEA3E0FF74081252AD8F048E33
:10324600057E017F08CDCCCD1200038E338F34AEC0
:1032560035AF36740CD39F74019E50030232EBA235
:10326600F9B3407EE5364535700375A382AE35AFBA
:103276003674016F4E700375A300AE35AF36740217
:103286006F4E700D9007B1E075F002A4FDACF08DA5
:10329600A3AE35AF3674036F4E700375A300AE351B
:1032A600AF367403BE00039F5013AC33AD34ED2F1D
:1032B600FFEC3EFE90006C125287E0F5A3AE35AFF0
:1032C60036EFB40B09EEB401057414125232AE3562
:1032D600AF36EFB40B07EEB4010375F80D7835126F
:1032E60052BD02325590003DE4F022753600753528
:1032F6000075F8099007B0E0FEA3E0FF7408BE0071
:103306001ED39F401A7E017F089007B0E0FCA3E021
:10331600FD1DBDFF011C1200038E338F34801F90EC
:1033260007B0E0FEA3E0FF74081252AD8F048E05CD
:103336007E017F08CDCCCD1200038E338F34AE359F
:10334600AF367411D39F74019E5003023421A2F943
:10335600B3500302341EE5364535700375A3D2AE6D
:1033660035AF3674016F4E700375A300AE35AF36B8
:1033760074026F4E700D9007B1E075F002A4FDACBB
:10338600F08DA3AE35AF3674036F4E700375A30090
:10339600AE35AF3674046F4E700375A300AE35AF0D
:1033A6003674056F4E700375A300AE35AF367406DE
:1033B6006F4E700375A300AE35AF3674076F4E704F
:1033C6000375A300AE35AF3674086F4E700375A350
:1033D60000AE35AF367408BE00039F5016AC33AD51
:1033E60034ED2FFFEC3EFE900067125287E5A3F006
:1033F60075A300AE35AF36EFB41009EEB40105740F
:1034060014125232AE35AF36EFB41007EEB40103E4
:1034160075F80D78351252BD0233442275360075A3
:10342600350075F809AE35AF367417BE0004D39F64
:1034360050030234FAA2F9B350030234F7E53645D5
:1034460035700375A3D2AE35AF3674016F4E700377
:1034560075A300AE35AF3674026F4E700D9007B18E
:10346600E075F002A4FDACF08DA3AE35AF36740363
:103476006F4E700375A300AE35AF3674046F4E7091
:103486000375A300AE35AF3674056F4E700375A392
:1034960000AE35AF3674066F4E700375A300AE35B9
:1034A600AF3674076F4E700375A300AE35AF367432
:1034B600086F4E700375A300AE35AF367408BE00B4
:1034C600039F500C900051125287E5A3F075A3009C
:1034D600AE35AF3674166F4E70057414125232AE96
:1034E60035AF3674166F4E700375F80D7835125277
:1034F600BD02342B2290003DE0B4AB0280030235BE
:103506009575360075350075F809AE35AF36741207
:10351600BE007CD39F4078A2F9B34070E5364535AE
:10352600700375A382AE35AF3674016F4E700375A6
:10353600A300AE35AF3674026F4E700D9007B1E042
:1035460075F002A4FDACF08DA3AE35AF3674036FF3
:103556004E700375A300AE35AF367403BE00039FED
:103566005009900056125287E0F5A3AE35AF367477
:10357600116F4E70057414125232AE35AF36741197
:103586006F4E700375F80D78351252BD0235102254
:10359600900046E4F074649007B0F8E4F0E8A3F015
:1035A60012342274C89007B0F8E4F0E8A3F0900053
:1035B6005DE0B4371A90005AE0900051F090005B3D
:1035C600E0900052F090005CE0900053F08046904E
:1035D60000467401F074659007B0F8E4F0E8A3F0D3
:1035E60012342274C89007B0F8E4F0E8A3F0900013
:1035F6005DE0B4371A90005AE0900051F090005BFD
:10360600E0900052F090005CE0900053F080067469
:1036160002900046F0900047E4F074669007B0F818
:10362600E4F0E8A3F012342274C89007B0F8E4F08E
:10363600E8A3F090005CE0B4371290005AE09000E6
:103646004BF090005BE0900054F080769000477459
:1036560001F074679007B0F8E4F0E8A3F0123422A2
:1036660074C89007B0F8E4F0E8A3F090005CE0B40A
:10367600371290005AE090004BF090005BE090000B
:1036860054F0803E7402900047F074689007B0F8DA
:10369600E4F0E8A3F012342274C89007B0F8E4F01E
:1036A600E8A3F090005CE0B4371290005AE0900076
:1036B6004BF090005BE0900054F08006740390009D
:1036C60047F022E55D2534FFAE3350010E900070C1
:1036D600125287E0F55EE55D2534FFAE3350010EEC
:1036E6000FBF00010E900070125287E0F55F8565EE
:1036F60061E55EB55F05855E5D8041E55FD3955EFC
:10370600401DE55FC3955E8560F0A4FFAEF0E56100
:103716008E048F05FF125242ED255EF55D801DE594
:103726005EC3955F8560F0A4FFAEF0E5618E048F01
:1037360005FF125242EDF404255EF55D22E55FD3E6
:10374600955E401DE55FC3955E8560F0A4FFAEF013
:10375600E5618E048F05FF125242ED255EF55D8010
:103766001DE55EC3955F8560F0A4FFAEF0E5618E52
:10377600048F05FF125242EDF404255EF55D22E545
:103786003875F00484FF7E008F5DE53875F004849B
:10379600ADF07C008D60756504753301753400E508
:1037A6005DC3943F50051236C980069001AFE0F51F
:1037B6005D855D53755200900042E075F020A4FFD0
:1037C600AEF09000C1E08E048F05FF1252428D5D6F
:1037D6009000A9E0D39538500302388B9000CDE0D5
:1037E600D395384010ED9001B0125292E0F5557520
:1037F6005400023888900098E0D395384043E55D40
:103806009001B0125292E0F55EE55D9001D0125241
:1038160092E0F55F9000CDE0F4042538F560900065
:1038260098E0FE9000CDE0F4042EF561E55EB55F0C
:1038360005855E5D8003123743855D5575540080AE
:1038460041E55D9001D0125292E0F55EE55D900192
:10385600F0125292E0F55F900098E0F4042538F5F6
:10386600609000A9E0FE900098E0F4042EF561E572
:103876005EB55F05855E5D8003123743855D5575D0
:1038860054000239329000D0E0D395385011E55DEE
:10389600900230125292E0F555755400023932907A
:1038A6000099E0D395385043E55D9002101252928C
:1038B600E0F55EE55D900230125292E0F55F900011
:1038C60099E0F4042538F5609000D0E0FE90009968
:1038D600E0F4042EF561E55EB55F05855E5D800367
:1038E600123743855D557554008041E55D9001F0C2
:1038F600125292E0F55EE55D900210125292E0F5EA
:103906005F9000A9E0F4042538F560900099E0FE88
:103916009000A9E0F4042EF561E55EB55F05855ECD
:103926005D8003123743855D55755400229000E192
:10393600E0F562756511753302753400AE25AF2664
:10394600E56275F00FA4FDACF0EDD39FEC9E40212F
:10395600E5628E048F05FF125242ED75F010A4FF4A
:10396600AEF0E53875F01184FD7C00ED2FF563802F
:103976000EE53875F01184FF7E00EF24F0F56385BF
:10398600635DE53875F01184AFF07E008F60123606
:10399600C9855D64AE25AF269000E1E075F00FA401
:1039A600FDACF0EDD39FEC9E4028753302753410C4
:1039B60085635D1236C985645E855D5FAE25AF267B
:1039C600E5628E048F05FF12527B8D60856261125F
:1039D6003743855D537552007555647554002290C2
:1039E60000E1E0F562756511753302753400AE25A8
:1039F600AF26E56275F00FA4FDACF0EDD39FEC9E0B
:103A06004021E5628E048F05FF125242ED75F010DB
:103A1600A4FFAEF0E53A75F01184FD7C00ED2FF5BC
:103A260063800EE53A75F01184FF7E00EF24F0F511
:103A36006385635DE53A75F01184AFF07E008F60B3
:103A46001236C9855D64AE25AF269000E1E075F0BB
:103A56000FA4FDACF0EDD39FEC9E402875330275A4
:103A6600341085635D1236C985645E855D5FAE255B
:103A7600AF26E5628E048F05FF12527B8D6085624C
:103A860061123743855D537552009000ABE0B40474
:103A960053E53875F00484FF7E008F5DE53875F0D8
:103AA6000484ADF07C008D60756504753301753452
:103AB60000E55DC3943F50051236C980069001AFFC
:103AC600E0F55DAE52AF53E55D12526074648E044C
:103AD6008F05FF125242AE52AF53EF2DFDEE3CFC66
:103AE6008C528D5375556475540022900076E0B45F
:103AF6000146E54075F00584FF7E008F5DE5407563
:103B0600F00584ADF07C008D60756505753305752F
:103B16003400E55DC3941750051236C9800690053A
:103B260087E0F55DAE54AF55E55D2FFF50010E748D
:103B3600641252AD8E548F55900077E0B40146E57D
:103B46004175F00584FF7E008F5DE54175F00584C3
:103B5600ADF07C008D60756505753305753448E5F7
:103B66005DC3941750051236C980069005CFE0F55F
:103B76005DAE54AF55E55D2FFF50010E74641252D1
:103B8600AD8E548F55900086E0B40249E543C39448
:103B96004175F00584FF7E008F5DE54375F0058471
:103BA600ADF07C008D60756505753306753400E5EE
:103BB6005DC3941350051236C98006900683E0F55E
:103BC6005DAE54AF55E55D2FFF50010E7464125281
:103BD600AD8E548F559000C8E0B402028003023CBB
:103BE60090E53875F01584FF7E008F5DE53875F039
:103BF6001584ADF07C008D607565157533037534DD
:103C0600F4E55DC3940B50051236C9800690046F27
:103C1600E0F55DE55D75F0FFA4FFAEF09000C9E04C
:103C26008E048F05FF125242ED90006BF0E53F7552
:103C3600F078A4FFAEF074FF8E048F05FF12524297
:103C46008C338D3474028C068D071252528F5DAC04
:103C560033AD347404FF12527B8D60756504753381
:103C66000675346EE55DC3941D50051236C980068F
:103C76009006FBE0F55DAE54AF55E55D2FFF5001B4
:103C86000E74641252AD8E548F552290007EE0B4AD
:103C960001179007B5E02555FFAE5450010E900070
:103CA600D2E01252AD8E548F5590007EE0B40316CA
:103CB600A201B3B3501090006AE0C39405A825B8DA
:103CC60000069526400280109000A0E02555FFAE24
:103CD6005450010E8E548F55900078E0B402028045
:103CE60003023EBE90007BE0602FE540D3941E4069
:103CF60028900014E0FEA3E0FF9000B6E075F00304
:103D0600A4FDACF0EFD39DEE9C400E9000DAE0A847
:103D160025B80005D395265003023EBE9000C3E0A9
:103D26008538F0A4FFAEF074051252607407125283
:103D3600528E338F34900082E0A825B80004952671
:103D46005012900083E075F002A4FDACF0EFC39D25
:103D5600EE9C4003023EBEE53875F00B84FF7E0004
:103D6600900600125287FEE0FFEE90007AE0FEEF2A
:103D76008E0088F0A4FFAEF074648E048F05FF12E7
:103D860052428C338D34900042E075F018A4FFAE99
:103D9600F09000C1E08E048F05FF1252428C068D12
:103DA60007900618125287AE33AF34E01252607491
:103DB600648E048F05FF1252428C338D34E53EA883
:103DC60033B80077D395344072E53EC39534FFE4AB
:103DD6009533FE8E338F347428BE00039F500C75C6
:103DE6003428753300740D900045F0AE33AF34902F
:103DF600007BE012526074288E048F05FF12524237
:103E06008C338D34AE52AF53740A8E048F05FF1275
:103E160052428D068C07AC33AD34CFCECF120003A1
:103E2600740A8E048F05FF1252428C338D34AE52C3
:103E3600AF531252B58E528F53807DE53EA833B8EC
:103E4600000495345072AE33AF34E53E1252AD8E57
:103E5600338F347428BE00039F500C753428753395
:103E660000740D900045F0AE33AF3490007BE01245
:103E7600526074288E048F05FF1252428C338D34A3
:103E8600AE52AF53740A8E048F05FF1252428D064E
:103E96008C07AC33AD34CFCECF120003740A8E0438
:103EA6008F05FF1252428C338D34AE52AF53EF2D35
:103EB600FDEE3CFC8C528D5322AE52AF53AC54AD4A
:103EC6005512000374648E048F05FF1252428C5201
:103ED6008D53900073E08C068D0712526074648EC9
:103EE600048F05FF1252428C528D53A2084017AE22
:103EF60025AF267405BE00039F5002D208E53AD3CB
:103F060094CC4002D2029000D5E0B402089000D7CB
:103F1600E0640160028017AE52AF53E5441252606E
:103F260074E78E048F05FF1252428C528D53900017
:103F360095E05402601B90008CE0A825B80012D3CF
:103F46009526400DA208B3B35007E53AC3949A40AC
:103F5600028028AE5BAF5C90008AE075F002A4FD9B
:103F6600ACF0EF2DFDEE3CFC74022DFD50010CE58E
:103F76003ABC0007D39D4003756901853A5C755BC1
:103F860000E56970030240159000E8E0C3956940BA
:103F960070E54075F00584FF7E009005701252872B
:103FA600E0F534753300AE33AF3490009AE0125228
:103FB6006074648E048F05FF1252428C358D3690E4
:103FC60000E8E004C395698C068D071252609000E4
:103FD600E8E08E048F05FF1252428C358D36900034
:103FE6008BE08C068D07125260740A8E048F05FFD3
:103FF600125242AE52AF53EF2DFDEE3CFC8C528D69
:104006005305699000E8E0C395695003756900900F
:104016000095E05401601B900089E0A825B80012C5
:10402600D39526400DA208B3B35007E538C394CC08
:1040360040028025900087E075F003A4FFAEF0E50E
:10404600662FFF50010E74032FFF50010EE538BE98
:104056000007D39F4003756A01853866E56A7003D9
:104066000240F09000E9E0C3956A4070E54075F0C3
:104076000584FF7E00900570125287E0F534753393
:1040860000AE33AF3490009AE012526074648E042E
:104096008F05FF1252428C358D369000E9E004C33D
:1040A600956A8C068D071252609000E9E08E048FA7
:1040B60005FF1252428C358D36900088E08C068DB5
:1040C60007125260740A8E048F05FF125242AE52D6
:1040D600AF53EF2DFDEE3CFC8C528D53056A9000DC
:1040E600E9E0C3956A5003756A0090009AE0A85209
:1040F600B800049553500990009AE0F553755200A4
:10410600229000D6E0B401028003024212A208B354
:1041160050030242109000A1E0B40168AE52AF53C2
:10412600AC25AD26120003743C8E048F05FF125297
:10413600429000B1E0BC00109D400D9000B3E0A895
:1041460052B8000495535002D203AE52AF53AC2579
:10415600AD26120003743C8E048F05FF1252429066
:1041660000B1E0C3940ABC0015D39D40119000B382
:10417600E0C39405A852B80005D3955350028002B7
:10418600C2038068AE52AF53AC25AD26120003744D
:10419600788E048F05FF1252429000B1E0BC0010E9
:1041A6009D400D9000B3E0A852B80004955350040A
:1041B600D2038038AE52AF53AC25AD26120003743D
:1041C600788E048F05FF1252429000B1E0C3940A24
:1041D600BC0015D39D40119000B3E0C39405A852CE
:1041E600B80005D3955350028002C203A203B34020
:1041F60019AE52AF539000B2E012526074648E044E
:104206008F05FF1252428C528D538002C2039000DA
:10421600D6E0B40258E53875F00884FF7E008F5D5D
:10422600E53875F00884ADF07C008D60756508751D
:1042360033017534E0E55DC3943F50051236C980FD
:104246000690026FE0F55DE55D75F05EA4FFAEF0E9
:10425600740A8E048F05FF1252428C568D577402D3
:10426600BC000AD39D4006755702755600A200B3DE
:104276004006A202B3B3500990001AE4F0A3F080FE
:1042860024AE52AF537400D39F74019E400C90002D
:104296001AE552F0A3E553F0800B74FF90001AF86C
:1042A600E4F0E8A3F09000B8E0D394024006A20838
:1042B600B3B34002800DAE52AF5374021252608EF9
:1042C600528F539000A1E0B4010DAE52AF53740269
:1042D6001252608E528F53AE52AF53745E125260BA
:1042E600740A8E048F05FF1252428C528D5374024B
:1042F600BC000AD39D400675530275520090001803
:10430600E552F0A3E553F022900042E090037012CC
:104316005292E0F567756864900042E0FE9000AC4A
:10432600E0D39E4037E53875F00884FF7E008F5D48
:10433600E53875F00884ADF07C008D60756508750C
:104346003303753496E55DC3941F50051236C98054
:1043560006900425E0F55D855D688035E53875F0E5
:104366000884FF7E008F5DE53875F00884ADF07C2B
:10437600008D607565087533037534B6E55DC394C5
:104386001F50051236C98006900445E0F55D855D2F
:1043960068229000E2E0F5627565117533047534A4
:1043A60000AE25AF26E56275F00FA4FDACF0EDD3A7
:1043B6009FEC9E4021E5628E048F05FF125242ED6E
:1043C60075F010A4FFAEF0E53875F01184FD7C00A1
:1043D600ED2FF563800EE53875F01184FF7E00EF52
:1043E60024F0F56385635DE53875F01184AFF07EE2
:1043F600008F601236C9855D64AE25AF269000E257
:10440600E075F00FA4FDACF0EDD39FEC9E4028754F
:10441600330475341085635D1236C985645E855D27
:104426005FAE25AF26E5628E048F05FF12527B8DA7
:1044360060856261123743855D6775686422900006
:10444600E2E0F562756511753304753400AE25AF8B
:1044560026E56275F00FA4FDACF0EDD39FEC9E400F
:1044660021E5628E048F05FF125242ED75F010A40D
:10447600FFAEF0E53A75F01184FD7C00ED2FF56393
:10448600800EE53A75F01184FF7E00EF24F0F563A7
:1044960085635DE53A75F01184AFF07E008F60129A
:1044A60036C9855D64AE25AF269000E2E075F00F53
:1044B600A4FDACF0EDD39FEC9E4028753304753413
:1044C6001085635D1236C985645E855D5FAE25AF76
:1044D60026E5628E048F05FF12527B8D6085626130
:1044E600123743855D677568649000DDE0B4047932
:1044F600900042E0FE9000ACE0D39E4037E5387570
:10450600F00884FF7E008F5DE53875F00884ADF015
:104516007C008D60756508753303753496E55DC35B
:10452600941F50051236C98006900425E0F55D8576
:104536005D688035E53875F00884FF7E008F5DE59F
:104546003875F00884ADF07C008D607565087533AC
:10455600037534B6E55DC3941F50051236C980064F
:10456600900445E0F55D855D6822900076E0B40133
:104576003BE54075F00584FF7E008F5DE54075F0F4
:104586000584ADF07C008D60756505753305753461
:1045960018E55DC3941750051236C9800690059F2D
:1045A600E0F55DE568255DC39464F568900077E005
:1045B600B4013BE54175F00584FF7E008F5DE54162
:1045C60075F00584ADF07C008D6075650575330565
:1045D600753460E55DC3941750051236C9800690A0
:1045E60005E7E0F55DE568255DC39464F568E56774
:1045F6002568F55A90007EE0B402109007B4E025D5
:104606005AFE9000D2E0F4042EF55A9000D5E0D37D
:1046160094014040E544C394E7501D74E7C39544B4
:10462600FE9007B6E08E00F5F0E884FF7E008F5D11
:10463600E55A255DF55A801CE544C394E7FE9007CC
:10464600B6E08E00F5F0E884FF7E008F5DE55AC384
:10465600955DF55AA2084006E5672464F55AE55AC1
:10466600D394644009E55AC39464F55A8003755A95
:10467600009000AEE0C3955A50069000AEE0F55AA1
:1046860022D2009000C4E0A825B800049526503B2D
:104696009000C4E0A825B8000495265003755A0F6B
:1046A6009000C4E004A825B8000495265003755A66
:1046B6000A9000C4E02402A825B8000495265005F7
:1046C600755A05C2007409900045F07E017F00907E
:1046D60000B4E01252609000C3E08E048F05FF1212
:1046E6005242E538BC000CD39D4008C200740A90C3
:1046F6000045F09000B5E0C39540500D9000C7E02E
:10470600A825B80006952640028008C200740B90C2
:104716000045F0A2004003755A0590007EE0B40300
:1047260006A201B3B34002802B90006AE0C3940551
:10473600A825B800049526500C90009FE0F55A7401
:104746000C900045F090006AE0A825B80004952674
:104756005002C200855A45900070E0255AFE90002E
:1047660042E075F01E84FC7F00EE2CF55A22900084
:1047760042E075F00584FF7E008F5D900042E07593
:10478600F00584ADF07C008D6075650575330375A5
:1047960034D69000C1E01475F00584FF7E00E55D17
:1047A600BE00039F50051236C9800BE55D90044696
:1047B600125292E0F55DE55D9007B7F09007B7E01D
:1047C600FE9000B0E0C39E50089000B0E09007B79E
:1047D600F022E54075F00584FF7E009005701252C8
:1047E60087E0F56CE56CD394644010E56CC3946483
:1047F60075F00F84FF7E008F6C8003756C0090004F
:1048060093E0256CF56C229007AAE0FEA3E0FF7406
:1048160004125252E538125260740F8E048F05FF4F
:104826001252429007A8ECF0A3EDF0900086E0B497
:104836000262E543C3944175F00584FF7E008F5DF7
:10484600E54375F00584ADF07C008D6075650575F2
:104856003306753414E55DC3941750051236C980C6
:1048660006900697E0F55D9007A8E0FEA3E0FF74CA
:104876000A8E048F05FF125242E55D8C068D0712E3
:104886005260740A8E048F05FF1252429007A8ECFC
:10489600F0A3EDF09007A8E0FEA3E0FF9007AEE0DE
:1048A600FCA3E0FDEDD39FEC9E400F9007AEE0F831
:1048B600A3E09007A8C8F0A3C8F02290008DE0B44A
:1048C600010385265090008DE0B402129000C3E0EB
:1048D6008538F0A4FFAEF074081252528F50900043
:1048E6008DE0B40303853A5090008DE0B40403854F
:1048F600405090008DE0B4050385415090008DE056
:10490600B4060385425090008DE0B40703854350FA
:1049160090008DE0B4080385445090008DE0B40902
:1049260003853F5090008DE0B40A03853E50900009
:104936008DE0B40B0385455090008DE0B40C0690D5
:10494600001BE0F55090008EE0FE90008FE0D39EB5
:10495600404B90008DE0B4041890008FE0C3955052
:104966005002D20490008EE0D395504002C20480DB
:104976002A90008EE0C39550500990008FE0D395A1
:104986005050028002D20490008EE0D39550500918
:1049960090008FE0C395505002C204802A90008E8A
:1049A600E0D39550400990008FE0C39550400280B7
:1049B60002C20490008EE0C39550400990008FE03B
:1049C600D395504002D20422900090E0B4010385B2
:1049D6002650900090E0B402129000C3E08538F0B3
:1049E600A4FFAEF074081252528F50900090E0B4BB
:1049F6000303853A50900090E0B40403854050903C
:104A06000090E0B40503854150900090E0B40603A1
:104A1600854250900090E0B4070385435090009083
:104A2600E0B40803854450900090E0B40903853F44
:104A360050900090E0B40A03853E50900090E0B498
:104A46000B03854550900090E0B40C0690001BE0E7
:104A5600F550900091E0FE900092E0D39E40409089
:104A66000091E0C395505009900092E0D3955050C4
:104A7600028002D206900091E0D395505009900032
:104A860092E0C395505002C206900090E0B401092E
:104A96009000CFE0D3953A50028002C206802A9059
:104AA6000091E0D395504009900092E0C3955040A4
:104AB600028002C206900091E0C395504009900022
:104AC60092E0D395504002D20622AE58AF5974F503
:104AD600D39F74019E400878581252BD024BEA7566
:104AE6005901755800AE25AF26E56CBE000DD39F63
:104AF60040099000A5E0D3956D40028023756D00B6
:104B0600E56CC39526F5509000A8E0D3956B400858
:104B1600E56B2550F56B80069000A8E0F56B8002EA
:104B2600056D900081E0D3953A401CE538C3953970
:104B36004015AE25AF26E56CBE00039F50099000D8
:104B4600A6E0D3956E4002806E9007B8E0A825B81F
:104B56000004952650037570009007B8E0A825B8A4
:104B6600000BD395264006E5269007B8F0E5707051
:104B760041E526C3956CF550E550D3940540037581
:104B860050059000A7E0C3956B5007E550C3956BA1
:104B960040028009E56BC39550F56B80069000A72F
:104BA600E0F56B9000A7E0D3956B40069000A7E078
:104BB600F56B756E008002056EE5707016900081CB
:104BC600E0C3953A500DE56C2405A825B800069576
:104BD600264002800F900094E0F56B7570017478A2
:104BE6009007B8F022AE58AF5974E9D39F74039E6C
:104BF600400878581252BD024D8975590175580002
:104C0600756B32A223402A756B19900094E075F0FB
:104C160002A4FFAEF0E56DBE0006D39F4002D2238C
:104C2600056D75700374789007B8F0756F00024DC6
:104C360078AE25AF26E56C6F4E7003024D78E56CB5
:104C4600BE000DD39F40099000A5E0D3956D4002AC
:104C5600800F756D00E570C394035003756B198062
:104C66000DE56CC39526F550E56D2550F56D900064
:104C760081E0D3953A400E9007B8E0A825B8000722
:104C8600D395264002800C056F900094E0B56F0323
:104C9600757000E570B40306A208B3B34002800A3B
:104CA600056FE56FB43C03757002E570B402299098
:104CB60007B8E0A825B8000ED395264009E526904A
:104CC60007B8F0756F00900081E0C3953A500975FA
:104CD6006F0074789007B8F0E570705A900081E024
:104CE600D3953A401CE538D395394015AE25AF2605
:104CF600E56CBE00039F50099000A6E0D3956E4078
:104D0600028008756E00756B4B8028E526C3956C8E
:104D1600F550E550D394054003755005900081E0A9
:104D2600D3953A4008E56E2550F56E8006E56E246B
:104D360006F56E756F00E5707016900081E0C395FC
:104D46003A500DE56C2405A825B8000695264002C4
:104D56008003757001E570B40118756B19056F90C5
:104D66000094E0B56F06757002756F007478900751
:104D7600B8F0E56B75F00AA4FFAEF09007B2EEF05E
:044D8600A3EFF02285
:095292002582F5825002058322F9
:0F008C0025E050020583258250020583F582226C
:10522100EF2F500205832582F582E5833E2EF5831B
:01523100225A
:1052AD00CFC39FFF50011E22C3EF9DFFEE9CFE2238
:09529B00E493F608740193F62275
:0852BD000806B60002180622E3
:0D526E00A3E004F07006120049E004F022F5
:0E003900A3E014F0B4FF06120049E014F02218
:0E525200048007C3CE13CECF13CFD5E0F622D3
:10514000BC000FBE0008ED8FF084FFADF022E4FE3E
:10515000FF22BE000DEF60FE54F0606F20E70302F7
:1051600051F6EAC0E0EBC0E078017A0075F001EE9C
:1051700020E710EF25E0FFEE33FE0AC5F023C5F06F
:1051800030E7F0EA5407F9096A7A007B0060010809
:10519000C3EC9E40167004ED9F4010ED9FFDEC9E09
:1051A000FCE5F0CA4ACA03F5F08005E5F003F5F026
:1051B000C3EE13FEEF13FFD9D77908CACBCAD8D0F4
:1051C000EAFEEBFFD0E0FBD0E0FA22EC8FF084FCAB
:1051D000ED54F045F0C48FF084FEEDC454F045F07A
:1051E000C48FF084FDEEC4FE54F02DFFEE540F3C4E
:1051F000FEADF07C0022790078008FF0EC7E082074
:10520000E70DC3CD33CD33C933C9C833C8DEF0840D
:1052100049F9E5F08FF0BE00E6FD7C00E9FFE8FE0D
:01522000226B
:0E526000F88FF0A4FFE5F0CE88F0A42EFE2219
:10000300EF8DF0A4F9A8F0EF8CF0A428F8EE8DF0B2
:06001300A428FEE9FF2213
:10523200600D782B02523C007830D8FED5E0F8227F
:10524200EEC0E07E00125140EFFDEEFCD0E0FE2207
:0C527B00EEC0E07E00125140D0E0FE22A8
:03001B0002001EC2
:0300530002005652
:03009B00020071EF
:030000000252A405
:0952A40075817175D000020685C8
:0B528700E5822FF582E5833EF58322CF
:0A0049000582D5820215831582227C
:10001E00C0E0C0F0C083C082C0D075D00012061000
:0B002E00D0D0D082D083D0F0D0E032E0
:10005600C0E0C0F0C083C082C0D075D000120613C5
:10006600D0D0D082D083D0F0D0E032C0E0C0F0C093
:1000760083C082C0D075D000120622D0D0D082D0E4
:0600860083D0F0D0E0324F
:00000001FF
